S01900006F70656E626C745F73746D3332663330332E7372656303
S3150800000000A00020FD040008D5040008D704000855
S31508000010D9040008DB040008DD040008000000001D
S31508000020000000000000000000000000DF040008D7
S31508000030E104000800000000E3040008E5040008E5
S315080000404D0500084D0500084D0500084D0500083A
S315080000504D0500084D0500084D0500084D0500082A
S315080000604D0500084D0500084D0500084D0500081A
S315080000704D0500084D0500084D0500084D0500080A
S315080000804D0500084D0500084D0500084D050008FA
S315080000904D0500084D0500084D0500084D050008EA
S315080000A04D0500084D0500084D0500084D050008DA
S315080000B04D0500084D0500084D0500084D050008CA
S315080000C04D0500084D0500084D0500084D050008BA
S315080000D04D0500084D0500084D0500084D050008AA
S315080000E04D0500084D0500084D0500084D0500089A
S315080000F04D0500084D0500084D0500084D0500088A
S315080001000000000000000000000000004D05000887
S315080001104D0500084D0500084D0500084D05000869
S315080001204D0500084D0500084D0500084D05000859
S315080001304D0500084D0500080000000000000000FD
S315080001404D0500084D0500084D0500080000000093
S315080001500000000000000000000000000000000091
S3150800016000000000000000004D0500084D050008CD
S315080001704D05000800000000000000000000000017
S30D08000180000000004D0500080F
S3150800018810B5054C237833B9044B13B10448AFF3BB
S3150800019800800123237010BDC8000020000000005D
S315080001A8E03B000808B5034B1BB103490348AFF306
S315080001B8008008BD00000000CC000020E03B0008D5
S315080001C803F016B903F023B908B54FF090431B6935
S315080001D8DB0703D400F050F8012008BD0020FCE72F
S315080001E830B5012887B013D04FF480540123CDE9E0
S315080001F801430025032301A94FF09040CDE9035395
S3150800020800F072FB2A4621464FF0904000F0A8FC01
S3150800021807B030BD70477047642000F003B800F097
S3150800022807B80000014B1880704700BFE40000209B
S3150800023810B50D4C02F0EEFE226890420ED30B4B19
S315080002480B4A18784FF4807148B9012018709161E3
S3150800025802F0E0FE074B1B881844206010BD0020FA
S3150800026818709162F4E700BFE8000020E600002055
S3150800027800100048E4000020024B4FF480729A628E
S31508000288704700BF00100048054B5A6902435A6177
S315080002985B6982B018400190019B02B0704700BFA5
S315080002A800100240264B1A6822F0070242F00202A2
S315080002B810B51A601A6802F00702022AFAD1214C08
S315080002C8236843F480232360236843F48033236038
S315080002D823689A03FCD5636823F4741343F4E81374
S315080002E86360E36A23F00F03E362236843F08073CD
S315080002F8236023689B01FCD5636823F0F0036360D9
S31508000308636823F4E06343F480636360636823F4F3
S3150800031860536360636823F0030343F00203636072
S31508000328636803F00C03082BFAD1074802F0F0F8C3
S31508000338002000F01BF9636823F48003636010BD8E
S31508000348002002400010024000A24A04BFB500F08F
S3150800035831F9FFF7A7FF18220021684603F034FC95
S315080003684FF48000FFF790FF124D4FF40030FFF767
S315080003788BFF4FF480774FF40010FFF785FF0024B2
S31508000388AF620223012669464FF090400493CDE9EF
S31508000398006401F043FA69462846CDE90076CDE9B6
S315080003A80244049401F03AFAFFF70AFFFFF70AFF36
S315080003B8FCE700BF001000480B4B9A6942F001029F
S315080003C89A619A6982B002F001020092009ADA6983
S315080003D842F08052DA61DB6903F080530193019B8E
S315080003E8072002B000F004B90010024010B5044610
S315080003F888B01422002103A803F0E6FB2268134BF1
S315080004089A4220D1124C636943F4003363616369E5
S3150800041803F400330193019B4FF4C0520223CDE93C
S31508000428032303210E23CDE906134FF0904003A9B1
S3150800043800F05AFAE36943F40003E361E36903F455
S3150800044800030293029B08B010BD00BF005C004081
S31508000458001002400268074B9A420AD1064AD36935
S3150800046823F40003D3614FF4C0514FF0904000F0D5
S3150800047801BB7047005C00400010024008B501F057
S3150800048875FA10484FF48073836201F05FF94FF0EC
S31508000498904001F05BF90C4B5A6922F400125A6134
S315080004A85A6922F400325A615A6922F480025A615A
S315080004B8DA6922F08052DA619A6922F001029A61B1
S315080004C808BD00BF00100048001002407047FEE74C
S315080004D8FEE7FEE7FEE770477047704700F07CB80E
S315080004E8034AD2F8883043F47003C2F88830704754
S315080004F800ED00E0DFF834D00D480E490E4A002317
S3150800050802E0D458C4500433C4188C42F9D30B4AB1
S315080005180B4C002301E013600432A242FBD3FFF719
S31508000528DFFF03F02DFBFFF711FFFEE700A0002011
S3150800053800000020C4000020AC3C0008C8000020C9
S31508000548E80E0020FEE7000010B5074B4FF0FF3213
S3150800055800241A611C61DA60DC609A629C62FFF703
S315080005688DFF204610BD00BF0010024038B50E4A60
S315080005780E4B054618784FF47A73B3FBF0F31068F8
S31508000588B0FBF3F000F07AF8044658B90F2D09D8ED
S31508000598024629464FF0FF3000F03CF8044B204647
S315080005A81D6038BD0120FCE700000020040000207B
S315080005B808000020074A08B5136843F010031360BB
S315080005C8032000F015F80020FFF7D0FFFFF7F4FE28
S315080005D8002008BD00200240034A044B11681B7816
S315080005E80B441360704700BF840C002004000020E9
S315080005F8074AD36823F4E0631B041B0C43F0BF6364
S31508000608000243F4003300F4E0600343D360704704
S3150800061800ED00E0174B70B5DC68C4F30224C4F19A
S315080006280705042D04F1040328BF04254FF0FF36F7
S31508000638062B06FA05F38CBF033C002421EA0303BC
S31508000648A34006FA04F422EA0404002843EA040349
S31508000658A8BF00F160404FEA0313BCBF00F00F00C3
S31508000668054ADBB2AABF00F56140135480F8003387
S3150800067870BD00BF00ED00E014ED00E00138B0F1F0
S31508000688807F0AD2064B074A5860F02182F8231061
S315080006980020072298601A6070470120704700BF3B
S315080006A810E000E000ED00E00B4AD36813F01003F1
S315080006B805D00A49CB6943F00203CB611023D268F7
S315080006C8520706D50549CA6942F00102CA6143F0CC
S315080006D80403014AD360704700200240880C0020B2
S315080006E8064B186910F0800007D0054A5A6002F1CF
S315080006F888325A601869C0F3C01070470020024053
S3150800070823016745034A136943F0800313610020F0
S31508000718704700BF00200240F8B5054602F082FC83
S31508000728104C07462646E368D9070FD4E3689A06A5
S3150800073844BF2023E360F368DB0603D4F06810F0AF
S31508000748040007D0FFF7B0FF012003E0681CEAD0D1
S315080007580DB90320F8BD02F065FCC01BA842E2D912
S31508000768F7E700BF002002402DE9F84F244C1E4643
S31508000778237E012B05460F4690463FD001234CF2AF
S3150800078850302376FFF7C8FFA0BB012D03D0022DF2
S315080007980CBF022504254FF00009DFF868A0CB46F0
S315080007A84FEA0913C3F12001A3F1200206FA01F161
S315080007B828FA03F3C4F81CB00B4326FA02F21343CB
S315080007C8DAF810209BB242F00102CAF810204CF25F
S315080007D8503027F81930FFF79FFFDAF8103023F062
S315080007E80103CAF8103028B909F101095FFA89F333
S315080007F89D42D5D800232376BDE8F88F0220FBE76B
S31508000808880C002000200240064B0022DA61064BBD
S315080008181A6942F004021A611A6942F040021A611A
S31508000828704700BF880C002000200240064B0022B3
S31508000838DA61064B1A6942F002021A6158611A69A6
S3150800084842F040021A617047880C002000200240D6
S315080008582DE9F041224D2B7E012B074688463DD0CF
S3150800086803680124A3422C764CF2503013D1FFF7C3
S3150800087853FF20B1012000232B76BDE8F081FFF74E
S31508000888C3FF4CF25030FFF747FF164A136923F0A7
S3150800089804031361EFE7FFF73FFF0028EAD14FF09B
S315080008A8FF33C8F8003020467E680E4CD7E9013277
S315080008B803EBC223B342DED93046FFF7B7FF4CF243
S315080008C85030FFF729FF236923F00203236110B18B
S315080008D8C8F80060CFE706F50066E7E70220CCE728
S315080008E8880C0020002002402DE9F74FD1F8008037
S315080008F8DFF87C915C4A002338FA03F402D103B086
S31508000908BDE8F08F012404FA03FC1CEA080500F088
S31508000918A0804C6824F0100A4FEA430E03260AF111
S31508000928FF3706FA0EF6012F6FEA060611D887680A
S3150800093807EA060BCF6807FA0EF747EA0B07876038
S31508000948476827EA0C0CC4F300179F4047EA0C07C8
S315080009584760C76807EA060C8F6807FA0EF747EA7A
S315080009680C07BAF1020FC76016D14FEAD30A00EB93
S315080009788A0A03F0070BDAF820704FEA8B0B4FF058
S315080009880F0C0CFA0BFC27EA0C0C0F6907FA0BF785
S3150800099847EA0C07CAF8207007683E4004F00307C0
S315080009A807FA0EFE4EEA06060660E60051D5D9F89D
S315080009B8186046F00106C9F81860D9F8186023F0D7
S315080009C8030707F1804706F0010607F58037019601
S315080009D803F0030E019EBE684FEA8E0E4FF00F0C09
S315080009E80CFA0EFCB0F1904F26EA0C0C33D01F4EC9
S315080009F8B04232D006F58066B04230D006F5806639
S31508000A08B0422ED006F58066B04214BF05260426E5
S31508000A1806FA0EF646EA0C06BE601668EF4314F4A4
S31508000A28803F0CBF3E402E431660566814F4003FBC
S31508000A380CBF3E402E435660966814F4801F0CBFC0
S31508000A483E402E439660D668A40254BF3E402E43C5
S31508000A58D660013350E70026DAE70126D8E70226EA
S31508000A68D6E70326D4E700BF00040140000400487F
S31508000A7800100240384A2DE9F04F00234FF0010ACA
S31508000A884FF00F084FF0030B31FA03F401D1BDE814
S31508000A98F08F0AFA03FC1CEA010452D023F0030576
S31508000AA805F1804505F5803503F00307AE68BF00F4
S31508000AB808FA07F9B0F1904F09EA060E43D0274E0F
S31508000AC8B04242D006F58066B04240D006F5806648
S31508000AD8B0423ED006F58066B0420CBF042605260D
S31508000AE8BE40764510D11668E44326401660566817
S31508000AF826405660966826409660D6683440D46084
S31508000B08AC6824EA0904AC605C0005680BFA04F4CE
S31508000B18E443DE08254000EB8606056003F0070572
S31508000B28376AAD0008FA05F527EA05053562C56886
S31508000B382540C560456825EA0C05456085682C404A
S31508000B4884600133A0E70026CAE70126C8E702261B
S31508000B58C6E70326C4E700BF0004014000040048AE
S31508000B680AB18161704781627047F0B5044687B05B
S31508000B78002851D090F8A93203F0FF021BB980F873
S31508000B88A822FFF733FC032384F8A932206800F06B
S31508000B983AFF00236568282601271846D9B28D42E8
S31508000BA803F101021BD8002328261946D8B2854224
S31508000BB803F1010321D804F110060FCE6D460FC5BF
S31508000BC833682B60231D0ECB206800F026FF002013
S31508000BD8012384F8240084F8A93207B0F0BD06FB7F
S31508000BE80143C3E90E0083F8297083F82810D986CB
S31508000BF883F82B0018641346D0E706FB004282F8F0
S31508000C08691182F8680182F86B11C2F87811C2F87E
S31508000C187C11C2F88011C9E70120DEE738B5044619
S31508000C2810B90125284638BD032380F8A93200687B
S31508000C3801F071F905460028F3D12046FFF70AFCAA
S31508000C4884F8A952EEE738B590F8A832012B04467D
S31508000C5810D0012580F8A852006800F0CBFE294676
S31508000C68204602F087FF206801F066F9002084F81C
S31508000C78A80238BD0220FCE790F8A832012B10B567
S31508000C88044610D0012380F8A832006800F0BBFE9D
S31508000C980021204602F06EFF206801F04FF9002077
S31508000CA884F8A80210BD0220FCE790F8A832012BA8
S31508000CB810B504460BD0012180F8A81202F05AFF95
S31508000CC8206801F039F9002084F8A80210BD02202E
S31508000CD8FCE790F8A832012B10B504460CD001237E
S31508000CE880F8A832002102F045FF206801F026F9AD
S31508000CF8002084F8A80210BD0220FCE790F8A82274
S31508000D08012A10B504460BD0012280F8A82284F8D7
S31508000D182410006801F00AF9002084F8A80210BD1A
S31508000D280220FCE72DE9F74F0446006801F008F9A8
S31508000D38020409D5DFF8DC97DFF8DC872068B0F805
S31508000D4844301F0400F19280206801F0F9F8430541
S31508000D580FD52268B2F8443023F480631B041B0CB1
S31508000D682046A2F8443002F0E7FD00212046FFF7A6
S31508000D78C5FF206801F0E4F8460408D52268B2F8E9
S31508000D88443023F480431B041B0CA2F84430206823
S31508000D9801F0D6F8850408D52268B2F8443023F459
S31508000DA800531B041B0CA2F84430206801F0C8F84D
S31508000DB8C0041CD52268B2F8403023F004031B048B
S31508000DC81B0CA2F84030B2F8403023F008031B0485
S31508000DD81B0CA2F84030204602F0D6FD2268B2F86D
S31508000DE8443023F480531B041B0CA2F844302068B3
S31508000DF801F0A6F8010517D52268B2F8403043F085
S31508000E080803A2F84030B2F8443023F400631B0400
S31508000E181B0CA2F84430B2F8403043F00403A2F899
S31508000E284030204602F09EFD206801F089F88205C8
S31508000E380BD52268B2F8443023F400731B041B0C44
S31508000E48A2F84430204602F072FD206801F078F8CE
S31508000E58C30508D52268B2F8443023F480731B0406
S31508000E681B0CA2F8443003B0BDE8F08FB0F8441064
S31508000E7889B211F00F0540F0B18011F0100103880E
S31508000E882AD109EA030343F400430380B0F8503033
S31508000E9894F8282003EBC20300EB4300E26BB0F892
S31508000EA80434C3F3090363641344E363204602F076
S31508000EB836FD94F82430002B3FF440AF226C002A04
S31508000EC87FF43CAF94F82430216843F08003A1F8F6
S31508000ED84C3084F8242031E79BB213F4006520D0FF
S31508000EE8B0F8503094F8682103EBC20300EB4303CB
S31508000EF8B4F86E21B3F80C34C3F30903C4F8843183
S31508000F0804F52C7101F0E8FA2268138823F07003B7
S31508000F181B051B0D43F080031380204602F0F0FCE6
S31508000F280CE71F047FF50AAF038823F070031B0537
S31508000F381B0D43F080030380B0F8503094F86821FD
S31508000F4803EBC20300EB4303B3F80C34C3F30903FA
S31508000F58C4F884318BB1D4F87C1171B1B4F86E2118
S31508000F6801F0BAFAD4F87C31D4F884211344C4F8C9
S31508000F787C312946204602F0C9FC2168D4F8785104
S31508000F88B1F8503001F20C409BB2BDB9C25A22F4EE
S31508000F98F8421204120CC252C25A48EA020292B223
S31508000FA8C2520B8823F4804323F0700383F440531A
S31508000FB843F4004343F080030B80BFE63E2D05D873
S31508000FC86A08EE0748BF01329202E8E76A09ED06A1
S31508000FD808BF02F1FF3248EA8222E0E72EB230F86B
S31508000FE82670BFB23A0440F1F78030F8263023F06D
S31508000FF870031B051B0D43F08003282120F82630B3
S3150800100801FB054100F5806E91F87431B3B9B0F863
S31508001018503091F86821063303EBC2033EF813A053
S31508001028CAF3090ABAF1000F00F0BA80B1F86E21BE
S315080010385346D1F87C1101F04FFAB1E091F86B31BB
S3150800104891F86821022B40F08980B0F850A0D1F8B1
S3150800105880314FEAC20C17F4804BD4443DD00CF1CA
S31508001068020C3EF81CA0CAF3090A9A4594BFA3EBDA
S315080010780A030023C1F88031282303FB0543D3F864
S3150800108880316BB930F8223023F4804323F070039B
S3150800109883F4005343F4004343F0800320F82230D6
S315080010A87B0610D5282303FB054393F8682130F8F7
S315080010B8223023F0F0031B051B0D43F4004343F0CD
S315080010C8C00320F82230BAF1000F69D0282101FBA5
S315080010D805415346B1F87021ABE70CF1060C3EF80A
S315080010E81CA0CAF3090A9A459CBFA3EB0A03C1F8D0
S315080010F880314FF0280303FB054388BFC1F880B148
S31508001108D3F880316BB930F8223023F4804323F0C2
S31508001118700383F4005343F4004343F0800320F834
S315080011282230790610D4282303FB054393F868214F
S3150800113830F8223023F0F0031B051B0D43F4004357
S3150800114843F0C00320F82230BAF1000F28D028212E
S3150800115801FB05415346B1F872216AE730F8223097
S3150800116823F0F0031B051B0D43F4004343F0C003AB
S3150800117820F8223091F868C10FFA8CF3082230F863
S31508001188233013F4804FB0F850305CD0023312FB8A
S315080011980C333EF813A0CAF3090ABAF1000F98D11E
S315080011A8282101FB0543D3F884215244C3F8842136
S315080011B8D3F87C215244C3F87C21D3F880211AB18C
S315080011C8D3F878319A4549D2282303FB05432046A4
S315080011D893F8681102F09AFB3A067FF5AFAD2068D6
S315080011E830F8263009EA030343F4004320F826308A
S315080011F806EB860604EBC60600F5806A96F82B30D9
S3150800120896F82810022B01D1FB053BD4B0F85030CC
S3150800121802334FF0280C03EBC1030CFB05473AF8D9
S3150800122813303A6CC3F309039A428CBFD21A0022C8
S315080012383A640CFB05473A6CC2B996F8281020465A
S3150800124802F06DFB7AE5063312FB0C333EF813A061
S31508001258CAF3090ABAF1000FA2D07BE701FB0541D8
S3150800126801F5B471206800F07FFEB5E7FA6B1A44F9
S31508001278FA637A6C05FB0CC113447B64214400F0BD
S3150800128873FE5BE5282202FB05420FFA81FE136C02
S31508001298B0F850B000934FEACE0C17F0400301930C
S315080012A807F48047DC4400F09A800CF1020C009B96
S315080012B83AF81CC0CCF3090C9C4534BFA3EB0C03C5
S315080012C800231364282303FB0543BFB21B6CABB981
S315080012D8204602F024FB002F00F09A8096F8281082
S315080012E8226832F8213023F0F0031B051B0D43F45E
S315080012F8404343F0800322F8213089E05FB130F893
S315080013082E3023F0F0031B051B0D43F4404343F02E
S31508001318800320F82E30282303FB054393F84C2036
S31508001328012A75D15A6CD96B9F6C62445A649A6BB8
S3150800133861449742D96322D3BF1A9F6496F82970E5
S3150800134893B2002F3ED1B0F850E096F828C000F2C4
S315080013580447774407EB0C17E2B93A8822F4F842AF
S315080013681204120C3A803A8848EA020292B23A8083
S31508001378282202FB05452A8E00F0E5FD48E01FB93C
S3150800138883F84C706246D9E7002283F84C209A64A1
S315080013983A46D3E73E2A0CD84FEA520CD20748BF3A
S315080013A80CF1010C4FEA8C2C1FFA8CFCA7F800C02C
S315080013B8DEE74FEA521CD20608BF0CF1FF3C48EAA2
S315080013C88C2CF1E7012FD3D1B0F850C096F82870C5
S315080013D800F20442624402EB07121380C8E70CF1D4
S315080013E8060C009B3AF81CC0CCF3090C9C4594BF24
S315080013F8A3EB0C03019B1364282303FB0543BFB225
S315080014081B6CBBB9204602F08AFA002F3FF466AF78
S3150800141896F82810226832F8213023F4E04323F09E
S31508001428400383F0300343F4004343F0800322F873
S31508001438213083E45FB930F82E3023F0F0031B051A
S315080014481B0D43F4404343F0800320F82E3028232D
S3150800145803FB054393F84C20012AD9D15A6CD96B5A
S315080014689F6C62445A649A6B61449742D96320D345
S31508001478BF1A9F6496F8297093B2002F3CD1B0F82A
S3150800148850E096F828C000F20C47774407EB0C178B
S31508001498D2B93A8822F4F8421204120C3A803A88E9
S315080014A848EA020292B23A80282202FB05456A8E69
S315080014B862E71FB983F84C706246DBE700229A6434
S315080014C883F84C203A46D5E73E2A0CD84FEA520C00
S315080014D8D20748BF0CF1010C4FEA8C2C1FFA8CFC7A
S315080014E8A7F800C0E0E74FEA521CD20608BF0CF17D
S315080014F8FF3C48EA8C2CF1E7012FD5D1B0F850C04B
S3150800150896F8287000F20C42624402EB0712138020
S31508001518CAE700BF0F8FFFFF0080FFFF11F0800F9B
S3150800152870B5044601F007054FF028001CD005FBE6
S3150800153800002118012048700A614A780D70CB709E
S3150800154802B1CD81022B04BF00230B7194F8A8328F
S31508001558012B13D0012384F8A832206800F072FA08
S31508001568002084F8A80270BD00FB054100FB054071
S31508001578002601F5B47180F86961DDE70220F2E713
S3150800158811F0800F10B501F0070204464FF0280342
S3150800159813D002FB0333C11801234B700A7094F861
S315080015A8A832012B13D0012384F8A832206800F04A
S315080015B88DFB002084F8A80210BD03FB020103FB7B
S315080015C80203002001F5B47183F86901E6E70220F1
S315080015D8F2E770B501F00701282606FB0104002585
S315080015E884F86811C4F87C21C4F88031C4F8845199
S315080015F884F8695104F5B471006800F0B5FC28460A
S3150800160870BD282301F0070103FB0101D1F8840105
S31508001618704770B501F00701282404FB0105C5E9E0
S315080016280F23AB6401EB810300EBC30301220026F9
S3150800163801FB044485F84C206E6483F8281083F867
S3150800164829200119006800F08FFC304670BD10B5D6
S31508001658044601F007006368984224D811F0800F01
S315080016684FF0280215D000FB0221631801225A7090
S3150800167801229A70187094F8A812914215D084F825
S31508001688A8221946206800F0E7FB002084F8A8027B
S3150800169810BD02FB014302FB0141002203F5B473A6
S315080016A881F86921E4E70120F2E70220F0E738B576
S315080016B8436801F00F029A42044626D811F0800FB3
S315080016C801F007024FF0280315D002FB0333C118AF
S315080016D801234B7000258D700A7094F8A832012BE7
S315080016E815D0012384F8A832206800F0D1FB84F8C5
S315080016F8A852284638BD03FB020103FB0203002053
S3150800170801F5B47183F86901E4E70120F2E70220DC
S31508001718F0E711F0800F18BF01F0070110B54FF078
S31508001728280415BF01FB044104FB0100401800F515
S31508001738B47099B21AB90273C180002010BD01228B
S315080017481B0C027301814381F7E70000B0F1904F43
S315080017580AD12C4B9A6A42F400329A629A6A22F49F
S3150800176800329A6200207047274B98420BD103F142
S31508001778784303F503339A6A42F480229A629A6A8E
S3150800178822F48022EDE7214B98420BD103F17843E6
S3150800179803F502339A6A42F400229A629A6A22F494
S315080017A80022DEE71A4B98420BD103F1784303F57A
S315080017B801339A6A42F480129A629A6A22F480126B
S315080017C8CFE7144B98420BD103F1784303F500335E
S315080017D89A6A42F400129A629A6A22F40012C0E7D8
S315080017E80D4B98420BD103F1784303F5FE339A6AF9
S315080017F842F480029A629A6A22F48002B1E70120CA
S31508001808704700BF0010024000040048000800485E
S31508001818000C004800100048001400482DE9F04F55
S3150800182802460D6895FAA5F44FF0010EB4FA84F449
S3150800183803264FF00F0C6FEA050835FA04F001D1B4
S31508001848BDE8F08F0EFA04F32B406CD04868471EA3
S31508001858012F1ED8976893FAA3F9B9FA89F993FA62
S31508001868A3FA4FEA490906FA09F927EA0909BAFA61
S315080018788AFA8F684FEA4A0A07FA0AF749EA070707
S315080018889760576808EA0709CF686F4349EA070760
S315080018985760D76893FAA3F9B9FA89F993FAA3FAB4
S315080018A84FEA490906FA09F927EA0909BAFA8AFA3A
S315080018B80F694FEA4A0A07FA0AF749EA07070228A0
S315080018C8D7601DD193FAA3F7B7FA87F7072FD1F888
S315080018D814A02ADCD2F820B093FAA3F7B7FA87F748
S315080018E893FAA3F9B9FA89F9BF000CFA07F74FEA88
S315080018F889092BEA07070AFA09FA47EA0A0717625B
S31508001908D2F8009093FAA3F7B7FA87F793FAA3F3EE
S31508001918B3FA83F37F0006FA07F75B0029EA070795
S31508001928984007431760013487E7D2F824B04FEA8E
S31508001938132999FAA9F7B7FA87F799FAA9F9B9FA0B
S3150800194889F9BF000CFA07F74FEA89092BEA07074E
S315080019580AFA09FA47EA0A075762D1E7024B1868EA
S31508001968C0F34000704700BF0010024007B51F4A81
S31508001978136843F001031360FFF7F0FF0128FBD152
S31508001988136823F0F80343F0800313604FF0FF331E
S3150800199801930199164B0B400193019B53605368B9
S315080019A813F00C0FFBD113680193019B23F0847382
S315080019B823F480330193019B1360106810F00070BC
S315080019C8FBD1136823F4802313604FF41F03506078
S315080019D8D06210630193019B93609060536A43F049
S315080019E88073536203B05DF804FB00BF0010024021
S315080019F80CC0FFF800234FF43F42A0F84430A0F883
S31508001A08402018467047B0F8403023F47C535B04EE
S31508001A185B0CA0F840300020704784B010B503ACC2
S31508001A2884E80E00BDE810400123A0F840300023E2
S31508001A38A0F8403004B0A0F84430A0F85030184652
S31508001A4870470000F0B50C7830F824200346C878AB
S31508001A5822F4EC4222F07002032803D8DFE800F0EB
S31508001A68444B4648012048F280052A4323F8242097
S31508001A780F78934C3EB233F8262022403A432A433D
S31508001A8823F826200D7B0A78002D40F08380CD8820
S31508001A984F786D0810266D0016FB023277B3B3F837
S31508001AA850603244A2F800540D7833F825205706BA
S31508001AB808D533F82520144044F4004444F0C004FB
S31508001AC823F82540CA780C78012A33F824107D4A69
S31508001AD802EA010218BF82F0200242F4004242F0EC
S31508001AE8800223F82420F0BD42F400720020BAE7E9
S31508001AF842F4C062FAE742F48062F7E7B3F8504066
S31508001B082244A2F808540A78B3F8504016FB023261
S31508001B180E69A4B202F20C4256BB155B25F4F845C9
S31508001B282D042D0C1553155B45F4004515530C78F3
S31508001B3833F8242052040BD533F8242022F0F00277
S31508001B481205120D42F4404242F0800223F824207E
S31508001B58097833F8212022F4804222F0700282F4B0
S31508001B68405242F4004242F0800223F82120BAE7A4
S31508001B783E2E06D87508F60748BF0135AD02ADB240
S31508001B88D4E77709F506504D08BF07F1FF3745EA48
S31508001B988725F4E712B233F82250254045F4014563
S31508001BA845F0800523F822500D78B3F850700E8951
S31508001BB8102212FB053505F58065BFB27608760052
S31508001BC8EE530D78B3F8506012FB05324D8902F5CD
S31508001BD88162B6B26D086D0095530A784D7812B2CF
S31508001BE8B5BB33F822506F0408D533F822502C4079
S31508001BF844F4404444F0800423F822400C7833F82F
S31508001C08242056060BD533F8242022F0F0021205B4
S31508001C18120D42F4004242F0C00223F824200D783F
S31508001C2833F8252022F4804222F0700248F2800414
S31508001C3882F44052224323F82520097833F82120D4
S31508001C4822F4E04222F04002144323F821404AE7EE
S31508001C5833F822506D0408D533F822502C4044F442
S31508001C68404444F0800423F822400C7833F82420B2
S31508001C7852060BD533F8242022F0F0021205120D6D
S31508001C8842F4004242F0C00223F82420CA780C78AD
S31508001C98012A33F824500B4A02EA050218BF82F0D3
S31508001CA8200242F4004242F0800223F824200978F0
S31508001CB833F8212022F0F0029204920C51E700BF73
S31508001CC88F8FFFFFBF8FFFFF0080FFFF10B50C7BCC
S31508001CD84A780B78BCBBF2B130F8232052060BD5EC
S31508001CE830F8232022F0F0021205120D42F40042C1
S31508001CF842F0C00220F823200A7830F8223023F070
S31508001D08C0031B051B0D43F4004343F0800320F86A
S31508001D182230002010BD30F8232054040BD530F8A3
S31508001D28232022F0F0021205120D42F4404242F036
S31508001D38800220F823200A7830F8223023F0F003AE
S31508001D489B049B0CDFE7002A44D130F82320520471
S31508001D580BD530F8232022F0F0021205120D42F4B2
S31508001D68404242F0800220F823200A7830F82230D0
S31508001D785C060BD530F8223023F0F0031B051B0D43
S31508001D8843F4004343F0C00320F822300A7830F8B9
S31508001D98223023F0F0031B051B0D43F4004343F0E0
S31508001DA8C00320F822300C7830F8243023F4804316
S31508001DB823F0700348F28002134320F82430097888
S31508001DC830F8213023F4E04323F040031A4320F87F
S31508001DD821209EE730F8232052040BD530F823201B
S31508001DE822F0F0021205120D42F4404242F0800237
S31508001DF820F823200A7830F822305B060BD530F80D
S31508001E08223023F0F0031B051B0D43F4004343F06F
S31508001E18C00320F822300A7830F8223023F0F0037D
S31508001E281B051B0D43F4404343F0800320F822307A
S31508001E380C7830F8243023F4E04323F0400348F2C2
S31508001E488002134320F82430097830F8213023F427
S31508001E58804323F07003B9E74B780A787BB130F8EA
S31508001E68223023F4E04323F0400383F0100343F4BD
S31508001E78004343F0800320F822300020704730F8EA
S31508001E88223023F4804323F0700383F48053EEE76B
S31508001E980B7B23BB4B780A781BB330F822305B06DA
S31508001EA80BD530F8223023F0F0031B051B0D43F43D
S31508001EB8004343F0C00320F82230CB78012B0ED01C
S31508001EC80A7830F8223023F4E04323F0400383F0FD
S31508001ED8200343F4004343F0800320F8223000200F
S31508001EE8704730F822305B040BD530F8223023F0DF
S31508001EF8F0031B051B0D43F4404343F0800320F809
S31508001F0822300A7830F8223023F4804323F070030D
S31508001F1883F44053DDE703460122A0F84020002059
S31508001F280322A3F84400A3F84020704711B9802378
S31508001F38A0F84C30002070470020704700207047F2
S31508001F48B0F84400704700EB4202013302F580629C
S31508001F585B0802EB83039A4200D1704731F8020BFB
S31508001F6822F8040BF7E70000F8B50C464978277BF2
S31508001F780129054640F08C812269A669616996425D
S31508001F8828BF1646F7B9B6B23346E288FFF7DBFF2D
S31508001F98B5F85010227805F204430B4403EB0213F4
S31508001FA81E80227835F8223023F4E04323F04003D4
S31508001FB883F0300343F4004343F0800325F82230C6
S31508001FC80020F8BDE3782778022B40F02A81236A97
S31508001FD89A4230F8272022F4F8724FEA02524FEA5A
S31508001FE8125280F00C8142F4014242F0800220F835
S31508001FF8272020789B1B236203B235F8232012F08A
S31508002008400FB3B262787ED0002A4DD1B5F8507029
S3150800201805F20C423A4402EB0012002E32D110881F
S3150800202820F4F8400004000C1080108840F40040A2
S31508002038108062892846FFF786FF226A2369616944
S3150800204860789A428CBF921B0023314486BF22626D
S3150800205832462362616193B2002848D1B5F85070B8
S31508002068267805F20440384400EB06103ABB028885
S3150800207822F4F8421204120C0280028842F4004242
S31508002088028025E03E2E06D87008F70748BF0130BB
S31508002098800280B2CCE77709F0069B4808BF07F1AB
S315080020A8FF3740EA8720F4E7012AC2D1B5F850700D
S315080020B805F20C423A4402EB00121380B9E73E2AAD
S315080020C80BD85608D70748BF0136B602B6B20680F7
S315080020D822892846FFF737FF63E75609D2068A4A50
S315080020E808BF06F1FF3642EA862292B2C8E70128F7
S315080020F8EED1B5F85060207805F20442324402EB76
S3150800210800121380E4E7002A4DD1B5F8507005F29D
S3150800211804423A4402EB0012002E32D1108820F409
S31508002128F8400004000C1080108840F40040108025
S3150800213822892846FFF707FF226A236961696078BA
S315080021489A428CBF921B0023314486BF22623246CC
S315080021582362616193B2002845D1B5F85070267894
S3150800216805F20C40384400EB06103ABB028822F404
S31508002178F8421204120C0280028842F400420280D5
S3150800218825E03E2E06D87008F70748BF01308002BA
S3150800219880B2CCE77709F0065B4808BF07F1FF3736
S315080021A840EA8720F4E7012AC2D1B5F8507005F24B
S315080021B804423A4402EB00121380B9E73E2A08D8CB
S315080021C85608D20748BF0136B602B6B206806289F3
S315080021D87FE75609D7064C4A08BF06F1FF3642EA92
S315080021E8862292B2CBE70128F1D1B5F8506020785B
S315080021F805F20C42324402EB00121380E7E742F478
S31508002208004242F0800220F82720B0F8507026785D
S3150800221800F204423A4402EB06129BB21380228962
S3150800222858E730F82720B0F85000B3B256064BBF27
S3150800223805F20C4205F20442121812184FEA07175B
S3150800224828464BBFD353D35362892289FFF77BFEAF
S31508002258637822786BB912B235F8223023F0F00386
S315080022681B051B0D43F4004343F0C00325F8223031
S3150800227897E6012B7FF495AE12B235F8223023F093
S31508002288F0031B051B0D43F4404343F08003EDE7B9
S31508002298002F3BD1A3692269B0F8500021789342F0
S315080022A886BF9B1AA3611A4605F20C43034498BFD6
S315080022B8A76103EB011352B91A8822F4F8421204EB
S315080022C8120C1A801A8842F400421A8008E03E2A3C
S315080022D810D85108D00748BF0131890289B2198038
S315080022E8227835F8223023F4804323F0700383F4E8
S315080022F840535FE65109D206034A08BF01F1FF3188
S3150800230842EA812292B2E0E70080FFFFE378022BD7
S3150800231876D1A1B9B0F85010227800F204430B44DC
S31508002328216903EB021300293BD11A8822F4F842E3
S315080023381204120C1A801A8842F400421A8062782B
S315080023482378002A51D1B5F8501005F20C420A44F0
S31508002358216902EB0313002935D11A8822F4F842B9
S315080023681204120C1A801A8842F400421A80E36989
S31508002378002BB5D0227835F8223044F240010B40BC
S315080023888B4201D0002BABD135F8223023F0F0036D
S315080023981B051B0D43F4004343F0C00325F8223000
S315080023A89EE73E2906D84A08CF0748BF0132920257
S315080023B892B2C3E74809CE06464A08BF00F1FF307D
S315080023C842EA8022F4E73E2906D84A08C90748BFE0
S315080023D80132920292B2C9E74809CA063D4A08BFBD
S315080023E800F1FF3042EA8022F4E7012ABFD1B5F8A6
S315080023F8501005F20C420A4402EB0313228AB5E789
S31508002408012B65D1A26923699A4295BF0023D21A7E
S31508002418A361A26198BF134691B9B0F85000217814
S3150800242805F20442024402EB011203BB118821F4A7
S31508002438F8410904090C1180118841F400411180FA
S3150800244861782278002938D1B5F8500005F20C4190
S31508002458014401EB0212E3B9138823F4F8431B0479
S315080024681B0C1380138843F40043138038E73E2B6C
S3150800247806D85908DF0748BF0131890289B2DEE75D
S315080024885809DE06134908BF00F1FF3041EA8021E2
S31508002498F4E73E2B07D85908D80748BF01318902FF
S315080024A889B211801CE75909DB060A4B08BF01F1F6
S315080024B8FF3143EA81239BB2D7E701297FF410AF9E
S315080024C8B5F8500005F20C41014401EB0212F2E797
S315080024D8012076E50080FFFF00EB4202F0B502F521
S315080024E880625D08084617462E46023036B9DB076D
S315080024F844BF32F8253001F81530F0BD37F8044BDB
S31508002508A4B200F8024C240A00F8014C013EECE794
S31508002518014B1860704700BF0000002008B580B15D
S31508002528D0F8B43213B10023C0F8B43209B1C0F8F0
S31508002538B012012380F89C32027001F02FFA0020AD
S3150800254808BD0220FCE7012310B580F89C32D0F8B4
S31508002558B43201795B6804469847204601F080FA48
S31508002568204601F061FA002010BD19B1C0F8B4126E
S31508002578002070470220704708B501F063FA00206A
S3150800258808BD08B5D0F8B4320BB9022008BD1B68D7
S3150800259898470028FAD0F8E708B5D0F8B4325B6847
S315080025A89847002008BD38B5044600F52A75284618
S315080025B800F0E0FA012394F8A812C4F89432B4F8A3
S315080025C8AE32C4F8983201F01F03012B0ED007D398
S315080025D8022B10D001F08001204601F06DFA03E0C5
S315080025E82946204600F0F6F8002038BD2946204638
S315080025F800F014FAF8E72946204600F034FAF3E71B
S3150800260870B50546164649BBD0F89432032B1ED139
S31508002618D0F86031D0F8642193420BD99B1A9A42B4
S31508002628C0F860318CBF9AB292B2314600F0F2FA1D
S31508002638002070BDD0F8B4321B6923B190F89C22EB
S31508002648032A00D19847284600F0ECFAF0E7052B4C
S31508002658EED1C5F8941201F02FFAE9E7D0F8B432AA
S315080026689B692BB190F89C22032A01D19847DFE78A
S315080026780220DEE770B5134604460E46002948D1FF
S31508002688D0F89422022A3DD1D0E90852954214D9A5
S31508002698AA1A0262194692B200F0B4FA33461A46E2
S315080026A81946204601F054FA94F8A032012B4FF047
S315080026B8000001D184F8A00270BDC369B3FBF2F526
S315080026C802FB153565B99A420AD8D0F8982293427A
S315080026D806D22A4600F096FAC4F898522B46DEE740
S315080026E8D4F8B432DB682BB194F89C22032A01D1BA
S315080026F8204698478021204601F0DEF9204600F05A
S315080027089CFAD1E732F00403CED1802101F0D4F93E
S31508002718CAE7D0F8B4325B6933B190F89C22032A29
S3150800272802D198470020C7E70220C5E770B50022FE
S315080027380446114601254026402301F09FF93346F1
S315080027488021C4F85851C4F864610022204601F073
S3150800275895F9D4F8B832A5610021666284F89C52C6
S31508002768C4F894126160C4F8A41223B1D4F8B43238
S3150800277820465B689847002070BD017400207047A2
S3150800278890F89C3280F89D32042380F89C32002009
S31508002798704790F89C32042B04BF90F89D3280F855
S315080027A89C320020704708B590F89C22032A04D169
S315080027B8D0F8B432DB6903B19847002008BD10B5D4
S315080027C88021044601F078F920460021BDE810402A
S315080027D801F072B937B50B7803F06003202B04466D
S315080027E80D4612D0402B10D0002B5BD14B78092B05
S315080027F858D8DFE813F0E90005015700FE0057002E
S31508002808840013005700D200A000D4F8B432294631
S315080028189B6820469847002003B030BD0023ADF8D2
S3150800282806304B881A0A013A062A3BD8DFE802F02E
S3150800283804202D3A3A525C00D0F8B0321B68207C46
S315080028480DF106019847BDF8062052B1EB8843B149
S315080028589A4228BF1A4601462046ADF8062000F0D7
S31508002868C4F9EB88002BD6D1204600F0DBF9D2E76D
S31508002878027CD0F8B43232B99B6A0DF10600984743
S3150800288802234370DFE7DB6AF7E7DBB2052B09D8D3
S31508002898DFE803F0030C1014181CD0F8B0325B6894
S315080028A8002BCCD12046FFF78AFFB4E7D0F8B03220
S315080028B89B68F5E7D0F8B032DB68F1E7D0F8B032B4
S315080028C81B69EDE7D0F8B0325B69E9E7D0F8B032B2
S315080028D89B69E5E7037C002BE4D1D0F8B4320DF107
S315080028E806005B6B9847AEE7037C002BDAD1D0F875
S315080028F8B4320DF106001B6B98470723C1E78B888E
S31508002908002BCFD1CB88002BCCD14D887F2DC9D8A9
S3150800291890F89C32032BC5D0E9B280F89E1201F0D4
S31508002928FBF8204600F07EF91DB1022384F89C3294
S3150800293871E70123FAE78978374D01292970B1D853
S3150800294890F89C32022B08D0032B14D0FFF737FFD8
S3150800295829782046FFF720FE5DE7002984D0012163
S315080029680323416080F89C322046FFF70AFE0228B6
S315080029787FF47AAF96E731B9022380F89C32416032
S31508002988FFF70AFE70E7416801293FF46DAFC9B23F
S31508002998FFF702FE29786160E6E7CA88012A81D12D
S315080029A890F89C32002B3FF47DAF022B04D9032BF9
S315080029B87FF478AF011D03E00146002341F8083F7C
S315080029C8204600F012F926E790F89C32013B022BC4
S315080029D83FF668AFCB88022B7FF464AF0123C36048
S315080029E8D0F8A4320BB10323C360022204F10C0108
S315080029F8E6E74B88012B7FF40EAFC4F8A43233E719
S31508002A0890F89C32013B022B3FF64CAF4B88012BC2
S31508002A187FF401AF0023F0E7EC00002038B50B7807
S31508002A2803F06003202B04460D4602D0402B00D045
S31508002A38ABB994F89C32013B022B10D82B79012BA1
S31508002A480DD8D4F8B43229469B6820469847EB88AF
S31508002A581BB910B9204600F0E5F8002038BD204615
S31508002A68FFF7ADFEF9E738B50A7802F06002202AC2
S31508002A7804460B4614D0402A12D06AB95A788D886B
S31508002A88012AE9B220D036D3032A05D190F89C2228
S31508002A98022A27D0032A0BD02046FFF790FE05E026
S31508002AA8D4F8B4221946926820469047002038BDC3
S31508002AB85A882AB94A0603D0DB880BB900F0FCFF06
S31508002AC8204600F0AFF8F1E790F89C22022A09D0D0
S31508002AD8032AE1D15B88002BE8D14D06F0D000F037
S31508002AE8F9FFEDE74B06D7D000F0E6FF8021204630
S31508002AF800F0E2FFDAE790F89C32022B18D0032B95
S31508002B08CAD101F00F02142315F0800F03FB020245
S31508002B181DD09269002ABFD001F07F0505FB033551
S31508002B28054411F07F031DD12B60022229460AE0CD
S31508002B384A06B1D12B064CBF00F1140100F5AA715B
S31508002B4800230B600222204600F04FF8AEE7D2F8C1
S31508002B585821002AA0D001F07F0503FB050505F5D5
S31508002B68AA75DEE7204600F0C3FF08B10123DBE7B4
S31508002B782860DAE70B7803704B784370CA788B7845
S31508002B8803EB022343804A790B7903EB02238380FC
S31508002B98CA798B7903EB0223C380704710B5802165
S31508002BA8044600F089FF20460021BDE8104000F0E1
S31508002BB883BF30B588B105462B1A15F8014BDBB229
S31508002BC8002CF9D101335B0013800B7003234B707B
S31508002BD80138022310F8015F05B930BD5A1CD2B274
S31508002BE8CD540233DBB28C54F4E710B513460222EF
S31508002BF8C0F89422C0E907330A46002100F09AFF74
S31508002C08002010BD08B513460A46002100F092FFB9
S31508002C18002008BD08B513460A46002100F098FFAB
S31508002C28002008BD08B50423C0F8943200231A46C4
S31508002C38194600F07FFF002008BD08B50523C0F82F
S31508002C48943200231A46194600F082FF002008BD70
S31508002C5872B6704762B67047FFF7FABF10B500F04C
S31508002C68A1F9C8B1FDF7B0FAB0B100F0FFFBFDF75E
S31508002C786BFC00F0A5F900F097F9084B20F06040C6
S31508002C8820F07F00986000F08FF94468FFF7E2FFAC
S31508002C982346BDE81040184710BD00BF00ED00E008
S31508002CA8F8B51446461A4FF6FF75013CA4B2AC426D
S31508002CB800D1F8BD0B788B554F1C00F000FC39463F
S31508002CC8F3E72DE9F8430546FDF70AFD002405F163
S31508002CD804082F6858F8046004EB070900F0EFFBAE
S31508002CE83246002349460220FDF73EFD60B9E359FE
S31508002CF8B3420BD10434B4F5007FEAD10124FDF7B9
S31508002D0801FD2046BDE8F8830024F8E70446F6E7FF
S31508002D1838B50E4B984204460D4607D00C4A9142E0
S31508002D2812D0FFF7CEFF10B904460BE0094C23680A
S31508002D389D4207D020464FF4007240F8045B2946A6
S31508002D48FFF7AEFF204638BD1C46F0E7F402002020
S31508002D5800400008F00000202DE9F0419846036875
S31508002D6821F4FF76013304460D46174626F0010678
S31508002D7806D140F8046B4FF400723146FFF790FF0E
S31508002D882368B34205D020463146FFF7C1FF0446FB
S31508002D98E8B123680435ED1A254406F50076B844E3
S31508002DA800F08DFB231DEB1AB3F5007F06D32046EA
S31508002DB83146FFF7ADFF044648B1051D17F8013B34
S31508002DC805F8013B4745EBD10120BDE8F081002015
S31508002DD8FBE70000034A4FF0FF331360024A13600B
S31508002DE8704700BFF0000020F402002030B40E4CF3
S31508002DF84D1E0B46211A8D4213D80C49884210D904
S31508002E08411E1944A1420CD820F4FF71084C21F040
S31508002E180101A142014630BC0CBF06480648FFF727
S31508002E289BBF002030BC7047FFFF0308FF3F000820
S31508002E3800400008F4020020F000002030B51D4DBF
S31508002E4885B04A1E2B1A00249A42009420D820F4EA
S31508002E58FF63194A23F00703934219D9421E0A4405
S31508002E68AA4215D80144C91AC1F3CF25C1F30A01E4
S31508002E7809B10135ADB20024CDE901430123039315
S31508002E88FDF72EFCA3B2AB4205D30124FDF73AFCA5
S31508002E98204605B030BD00F012FB694601A8FDF7CB
S31508002EA8D7FC013420B9029B03F500630293E9E7CE
S31508002EB80024EBE7FFFF0308FF3F000807B50F4AA2
S31508002EC81368013317D0D2E901310B44D1680C488D
S31508002ED80B4411690B4451690B449169D2690B4437
S31508002EE8134402AA5B4242F8043D0421FFF77EFF19
S31508002EF803B05DF804FB0120FAE700BFF4020020DE
S31508002F08884100080D4B0E4A1B68126813440D4A7F
S31508002F18126813440C4A126813440C4A126813447C
S31508002F280B4A126813440B4A126813440A4A126871
S31508002F38D3420CBF01200020704700BF004000089C
S31508002F4804400008084000080C4000081040000823
S31508002F581440000818400008884100080A4808B5BF
S31508002F680368013305D109480368013306D10120EE
S31508002F7808BDFFF7A6FE0028F5D1F9E7FFF7A1FE79
S31508002F88003018BF0120F3E7F4020020F000002003
S31508002F980048704700400008FFF71CBFFFF726BF28
S31508002FA8FFF74CBFFFF7AEBFFFF7F2BF08B5FFF74D
S31508002FB885FF18B1BDE80840FFF7D0BF08BD000077
S31508002FC8024B00221A605A609A60704710E000E0C7
S31508002FD808B5FFF7F5FF054B054A5A600521002293
S31508002FE89A601960034B1A6008BD00BF10E000E03C
S31508002FF83F190100F8040020044B1B68DB0341BF96
S31508003008034A136801331360704700BF10E000E0F5
S31508003018F804002008B5FFF7EFFF014B186808BD4C
S31508003028F804002008B5FFF7E7FF014B186808BD44
S31508003038F8040020012838B504460D4604D94FF48B
S31508003048DE710E4800F088F90D49182060430B1800
S315080030585C7C1A7C94420ED0DA6815705A7C5C68D7
S3150800306801325A74DA680132A242DA6001D90A587A
S31508003078DA60012000E0002038BD00BFF83B0008F0
S315080030883C050020012870B505460E4604D94FF4BC
S31508003098EF710D4800F060F90C4C18226A43A31822
S315080030A8587C80B1996809783170597C5868013913
S315080030B8597499680131814288BFA25899604FF0BE
S315080030C8010088BF9A6070BDF83B00083C050020DF
S315080030D81E4B1F4903F1180210B5481C5A614024B3
S315080030E800220A70C3E902001860081919491C82E7
S315080030F80A6019491C850124586083F82A40481C27
S315080031080C70164C9861C3E9080001F14000D861B3
S31508003118DA629A7412492046FFF700FA11492046DE
S31508003128FFF723FA2046FFF727FAD4F8C002FDF777
S31508003138BCFD00F03DF9B0F5FA6F05D24FF4FA6018
S31508003148BDE8104000F02EB910BD00BF3C050020B0
S31508003158700500206C050020B1050020F405002044
S31508003168740000201000002010B5054CD4F8C002E1
S31508003178FDF7AFFD2046BDE81040FFF7E4B900BFEC
S31508003188F40500203F292DE9F04107460C4603D9E6
S31508003198B521134800F0E0F8124D21462878FFF7C4
S315080031A849FF012803D0B9210D4800F0D5F8DFF802
S315080031B830803E46A4B2F31B9BB2A34201D3BDE8B6
S315080031C8F08100F07CF916F8011B2878FFF732FF22
S315080031D80128F0D0C221404600F0BEF8EBE700BF50
S315080031E8F83B0008700500202DE9F8431E4B1F4ED2
S315080031F81F4D8046D3F8C0020F46FDF793FD347875
S315080032081C4B8CB929461878FFF73CFF012803D0D0
S3150800321800242046BDE8F8832B78013B3E2BF7D8D7
S31508003228154B30701C70F4E7DFF84C90187899F84D
S31508003238001001312944FFF725FF01280446E7D184
S3150800324899F800302A780133DBB29A4289F80030B7
S31508003258DED1691C4046FFF723FD0023337099F831
S3150800326800303B70D5E700BFF4050020F8080020B9
S31508003278B8080020B1050020F90800202DE9F34117
S31508003288184E3478012C04D94FF4FF71164800F00B
S3150800329863F8164B182202FB0434647CFCB1402CF4
S315080032A8DFF84480124F28BF402400250DF1070196
S315080032B83078FFF7E7FE012804D04FF4A17140469D
S315080032C800F04AF89DF80730EB550135EBB29C42F9
S315080032D8ECD82346064A0748812100F02BFC02B0A1
S315080032E8BDE8F08170050020F83B00083C05002081
S315080032F8FC040020F40500202DE9F041044600F0FE
S3150800330881FA214605461148114FDFF8488000F032
S315080033182DFC2C4686B2631B9BB29E4209D800F048
S3150800332871FA4023024601210848BDE8F04100F039
S315080033380FBC14F8011B3878FFF77CFE0128EAD081
S315080033484FF4B271404600F007F8E4E7F4050020A8
S31508003358B1050020F83B000808B500F0B0F8FCE70E
S3150800336810B500F0A3F8012814D00B4C2378012BCC
S3150800337810D1FFF74FFE094B094A1B681268134418
S3150800338803F5FA73984205D300232370BDE8104065
S31508003398FFF764BC10BD00BF00090020FC08002028
S315080033A804090020014B1860704700BFFC0800207C
S315080033B8014B1868704700BFFC08002008B5044B85
S315080033C81B78012B03D1FFF725FE024B186008BDB1
S315080033D8000900200409002008B5044B01221A70C8
S315080033E8FFF7ECFFBDE80840FFF7BABF0009002061
S315080033F808B5FFF731FC00F060F8FFF7E9FDFFF7BD
S31508003408CBFD00F00FF8BDE80840FFF7E5BF08B5A3
S3150800341800F055F8FFF7F0FD00F010F8BDE8084091
S31508003428FFF79EBF08B500F057F8FFF751FE024BA5
S3150800343802221A7008BD00BF0C00002007B509480B
S315080034480DF10701FFF7D0FE012807D1064B9DF8B5
S315080034580710044802221A7000F05AF803B05DF8FB
S3150800346804FB00BF080900200C000020FFF77CBEFB
S3150800347808B5054B1B78022B02D1C9B2FFF782FEA5
S31508003488BDE8084000F03CB80C000020044B1B7847
S31508003498013BDBB2022B9ABF024AD05C4020704738
S315080034A80C000020343C0008FFF7F0BF08B500F010
S315080034B81FF8003018BF012008BDFCF7ADBEFCF7A1
S315080034C8AEBE0000034BFE22DA7002221871A3F87A
S315080034D84420704748090020044B00229A6483F860
S315080034E84320A3F844201A809A7070474809002098
S315080034F8024B1878003018BF012070474809002089
S31508003508024B002283F84320704700BF4809002071
S31508003518F8B503787E4CFF2B05462CD1E3701023AB
S3150800352801252371002363712580FFF7AFFFA0717A
S31508003538FFF7BAFFE071FFF7B7FF0823000A207202
S315080035486572A572A4F84430FFF726FD94F843304F
S31508003558012B02D11020FFF7B5FFB4F94410002952
S3150800356840F3D480012384F8433089B26948BDE81A
S31508003578F840FFF77DBF2678012E40F0C780F32B69
S3150800358858D01FD8CF2B00F0BE8007D8C92B00F01B
S315080035988380CC2B00F08980202030E0D12B00F0E6
S315080035A8AB80C0F08C80D22BF6D10025FF23E370C0
S315080035B825716571FFF76AFFE571A0712572657255
S315080035C807232BE0FA2B4CD00BD8F52B11D028D390
S315080035D8F62BE1D1FF23E3704368A364A4F844609B
S315080035E8B4E7FD2B49D0FE2B51D0FC2BD4D10020B3
S315080035F805E0FFF74BFF6A78904203D82220FFF7C9
S3150800360861FFA3E7A16C201DFFF74AFBFF23E370C0
S315080036186A78A36C1344A3646B780133A4F844301E
S3150800362894E7FFF733FF6B788342E7D26968A164AA
S315080036386A78E8E7FF23E370A66C476800253744ED
S31508003648BE4207D10123A3800023C4F80750A371FB
S315080036580823E3E716F8013B1D44EDB2FFF72FFFF1
S31508003668EEE7FF23E3702C4BA364002323716371F1
S31508003678A3710723C4F80730EAE7FF23E3706278E3
S31508003688627100232371E38023720623C6E70023A9
S315080036982380FF23E370A1E7A76CFFF7F7FE6A1CF0
S315080036A8411E3846FFF77AFC08B93120A7E7FF23F9
S315080036B8E370FFF7EBFEA36C013803448DE7FFF7C9
S315080036C8E5FE6B780138984298DDFF23E370A4F885
S315080036D84460697829B9FFF769FC00287FF436AF92
S315080036E8E3E7AA1CA06CFFF759FC0028DDD06A7826
S315080036F8A36C1344A36429E74168A06CFFF750FC40
S315080037080028C6D1D1E7FFF7A9FAC2E7F8BD00BF76
S31508003718480900204B090020373C0008202303806D
S3150800372800487047480000200A230380004870476D
S315080037386800002008B590F89C32032B01D1FFF7E2
S315080037489DFD002008BD08B5FFF798FD002008BDB7
S3150800375808B50846FFF7D0FD002008BD10B5812139
S31508003768044600F09BF90121204600F097F900204D
S3150800377810BD000010B5402304460222812100F03E
S315080037887DF9402302220121204600F077F94023DB
S31508003798034A0121204600F0DBF9002010BD00BFCE
S315080037A8A80C002010B50A7812F0600F044612D14A
S315080037B84A780A2A14D00B2A15D0062A0BD14A8821
S315080037C8120A212A09D1CA880B49172A28BF17229B
S315080037D82046FFF70AFA002010BD08491722F7E71E
S315080037E801220749F5E78B7813B9054A1360F2E70A
S315080037F8FFF7D4F9EFE700BF5A0000205100002070
S315080038089409002000487047A80C002012230B8052
S31508003818004870479000002004230B800048704732
S31508003828A4000020002370B51E46050FECB2092D2A
S3150800383894BF3034373401F8134001EB430401339D
S315080038486670DCB2A2424FEA0010EED870BD0000DE
S315080038581A2310B50B80094B186808331B68C0185B
S315080038680AD0074B07491C680822FFF7DBFF042222
S3150800387805492046FFF7D6FF044810BDACF7FF1FD9
S31508003888B0F7FF1FAA000020BA000020A8000020F1
S3150800389810B5044C04480A462146FFF78AF920461B
S315080038A810BD00BFE80C00205D3C000810B5044CAC
S315080038B804480A462146FFF77CF9204610BD00BF92
S315080038C8E80C00206A3C000810B5044C04480A466F
S315080038D82146FFF76EF9204610BD00BFE80C002008
S315080038E83F3C000810B5044C04480A462146FFF731
S315080038F860F9204610BD00BFE80C0020473C0008C8
S3150800390800F52C71D0F8E802FEF74DBE282303FB14
S315080039180103D0F8E802D3F87C21FEF771BE282304
S3150800392803FB0103D0F8E802DA6BFEF7A3BED0F86A
S31508003938E802FEF738BF00008368022B10B5044674
S3150800394803D08E210648FFF707FDD4F8E8020121BF
S31508003958FEF713FFD4F8E802BDE81040FEF7E6BE06
S31508003968813C000810B50446FCF754FCD4F8E80274
S31508003978FEF706FFA36923B1024A136943F0060353
S31508003988136110BD00ED00E008B5D0F8E802FEF7AF
S3150800399800FFBDE80840FCF73EBC000010B51F4A0A
S315080039A804461F480823C0E900230223C0F8E84252
S315080039B883600361C4F8C002002383610362FDF7CC
S315080039C8D4F820B140F21B111648FFF7C5FC0022AF
S315080039D811461823D4F8C002FDF79BFE5823002287
S315080039E88021D4F8C002FDF794FEC0230022812165
S315080039F8D4F8C002FDF78DFE4FF488730022012122
S31508003A08D4F8C002FDF785FE4FF4807300228221A0
S31508003A18D4F8C002FDF77DFE002010BD005C00400A
S31508003A2898090020813C000808B5D0F8C002FDF7BF
S31508003A38F5F8032896BF024B0220185C08BD00BF9C
S31508003A487D3C000808B5D0F8C002FDF7FCF8032845
S31508003A5896BF024B0220185C08BD00BF7D3C0008D3
S31508003A6808B5D0F8C002FDF707F9032896BF024B38
S31508003A780220185C08BD00BF7D3C000810B51C462E
S31508003A88D0F8C00213462246FDF748FD032896BF1C
S31508003A98014B0220185C10BD7D3C000808B5D0F81B
S31508003AA8C002FDF76DFD032896BF024B0220185C7D
S31508003AB808BD00BF7D3C000808B5D0F8C002FDF770
S31508003AC8C6FD032896BF024B0220185C08BD00BF36
S31508003AD87D3C000808B5D0F8C002FDF7E8FD0328C4
S31508003AE896BF024B0220185C08BD00BF7D3C000843
S31508003AF811F0800FD0F8C0024FF028021DBF01F060
S31508003B087F0303FB0221091802FB010114BF887809
S31508003B1891F86A017047000008B5D0F8C002FDF7A9
S31508003B28EDF8032896BF024B0220185C08BD00BFB3
S31508003B387D3C000808B5D0F8C002FDF76AFD0328E1
S31508003B4896BF024B0220185C08BD00BF7D3C0008E2
S31508003B5808B5D0F8C002FDF73CFD032896BF024B0E
S31508003B680220185C08BD00BF7D3C0008D0F8C002DA
S31508003B78FDF747BD01290CBF08460020FCF730BBF6
S31508003B8870B50D4E0D4CA41BA4100025A54209D1ED
S31508003B980B4E0C4C00F020F8A41BA4100025A542D7
S31508003BA805D170BD56F8253098470135EEE756F821
S31508003BB8253098470135F2E7A43C0008A43C0008DC
S31508003BC8A43C0008A83C000802440346934200D1D6
S31508003BD8704703F8011BF9E7F8B500BFF8BC08BC3D
S31508003BE89E467047F8B500BFF8BC08BC9E467047A5
S31508003BF8433A2F576F726B2F736F667477617265C6
S31508003C082F4F70656E424C542F5461726765742F36
S31508003C18536F757263652F41524D434D345F535444
S31508003C284D333246332F7573622E6300003F004FBB
S31508003C3870656E424C540044656661756C7400572D
S31508003C48696E5553422042756C6B20496E746572CD
S31508003C5866616365004F70656E424C5420557365FE
S31508003C68720057696E5553422042756C6B2044653D
S31508003C787669636500000201022E2E2F5553425FAE
S31508003C884445564943452F5461726765742F7573C1
S31108003C9862645F636F6E662E63000000B6
S30908003CA4AD01000858
S30908003CA88901000878
S31508003CAC00127A0001000000100000000400000059
S31508003CBC7D37000865370008AD370008000000009E
S31508003CCC000000004F370008593700083D37000838
S31508003CDC0000000000000000000000002537000866
S31508003CEC000000003137000809022000010100C05D
S31508003CFC320904000002FF0000000705810240009B
S31508003D0CFF070501024000FF0A06100100000040EB
S31508003D1C01000000153800082138000899380008F9
S31508003D2CB538000859380008D1380008ED380008AD
S31508003D3C1201100100000040501DAC600001010288
S31508003D4C03010000040309041A0300000000000024
S31508003D5C0000000000000000000000000000000049
S30908003D6C0000000045
S705080004FDF1
